:02000000F8C046
:0200120011C318
:0200160022C105
:02001A0047C1DC
:14002600280900010302060705040405070602030100010359
:14003A00020604040602030100202020202020202020303016
:14004E003030302020202020202020202020202020202020EE
:1400620020904040404040404040404040404040400C0C0CF6
:140076000C0C0C0C0C0C0C404040404040400909090909092C
:14008A0001010101010101010101010101010101010101014E
:14009E004040404040400A0A0A0A0A0A020202020202020282
:1400B200020202020202020202020202404040402000000002
:1400C600000000000000000000000000000000000000000026
:1400DA00000000000000000000000000000000000000000012
:1400EE000000000000000000000000000000000000000000FE
:140102000000000000000000000000000000000000000000E9
:140116000000000000000000000000000000000000000000D5
:14012A000000000000000000000000000000000000000000C1
:14013E00000000000000000D0A416C746974756465203D20DD
:1401520025640D0A000D0A53657269616C2D746F2D50617222
:14016600616C6C656C20416C74697475646520456E636F6416
:14017A00657220436F6E7665727465722C2076657273696FDE
:14018E006E20312E30322C20393630302C4E2C382C310D0AA1
:1401A200003C696E7465676572206F6E6C79207072696E74F0
:1401B6002C20757365202D6C66703F3F20746F2072656C69C0
:1401CA006E6B3E00286E756C6C207074722070617373656411
:1401DE002900616263646566003000616263646566003000DA
:1401F200CFE5D4E0CDBFDEBFC052D0400AEA08830024EFE0D4
:14020600F1E011E0EE33F10711F00192FBCF0083E3E4F1E090
:14021A00A0E6B0E011E0E23FF10721F0C89531960D92F9CF14
:14022E00E6D0FFCF97D71801232C332420BC09B988E98AB9B9
:1402420086E880BD44274093190140931A0140930F01409301
:14025600100187D708952A920A932A933A938A939A93EA93DE
:14026A00FA932FB62A920CB120911A012F5F277020931A01D6
:14027E0020901901221501F48BE191E0E22FFF27E80FF91F53
:14029200008329902FBEF991E99199918991399129910991C9
:1402A600299018952A923A920A931A938A939A93EA93FA93B8
:1402BA002FB62A9220900F0130901001321479F000910F01AE
:1402CE000F5F077000930F0181E191E0E02FFF27E80FF91F7D
:1402E20020802CB801C0559829902FBEF991E99199918991E8
:1402F600199109913990299018952090190130901A01321496
:14030A00D1F3009119010F5F0770009319018BE191E0E02FF2
:14031E00FF27E80FF91F008108951CD7409110014F5F47703E
:1403320020900F014215E1F381E191E0E42FFF27E80FF91FB1
:14034600008340931001559A0CD708952090190130901A0128
:14035A00321419F001E010E002C000271127089512D722970F
:14036E008CEF81BB442755271BC08CEF82BB66277727798323
:1403820068836F5F7F4F6436E0E07E07C4F382B3837082BBE5
:1403960066277727798368836F5F7F4F6436E0E07E07C4F30F
:1403AA004F5F5F4F4017510714F3442755271BC083E082BBCB
:1403BE0066277727798368836F5F7F4F6436E0E07E07C4F3E7
:1403D20082B3837082BB66277727798368836F5F7F4F64366A
:1403E600E0E07E07C4F34F5F5F4F4017510714F32296AED6B9
:1403FA000895442764E770E0AB018FE388BB87BB8FE185BBF9
:14040E0084BB80EE82BB81BB85E083BF222422BE07E610E00A
:1404220007DF7894AB9AAC9A89B7816089BF07C0FA0101918C
:14043600AF0177DF0AE010E095DFFA0120802220A9F70EC013
:14044A000FD0B8010F3FEFEF1E0739F09BD0AB9A89B78160BB
:14045E0089BFAC9801C0AC9AF1CF08959BD626978FEF9FEF60
:140472005C0166277727CC247DC041DF11277ED8E02E0D30C8
:1404860011F40AE04EDF0E2D4CDF4C2D552740304507B1F08E
:14049A004130E0E05E07D9F04230E0E05E0701F14330E0E033
:1404AE005E0729F14430E0E05E0751F14530E0E05E0709F449
:1404C20043C058C08E2D813419F4CC24C39452C086E0C82ED9
:1404D6004FC08E2D8C3419F482E0C82E49C086E0C82E46C0B8
:1404EA008E2D843519F483E0C82E40C086E0C82E3DC08E2D10
:1404FE00803219F484E0C82E37C086E0C82E34C00E2D112717
:140512000BD80030010731F46030670791F48E2D8D3279F42B
:14052600CE01FB01E80FF91FE082CB010196BC016530E0E010
:14053A007E07E1F485E0C82E19C086E0C82E16C08E2D8D3075
:14054E0089F422242D828E01A7D658010035EBEF1E072CF072
:140562008CEE97E7801791071CF48FEF9FEF5C0186E0C82E89
:140576008C2D863009F07FCF950102E610E010D88501269623
:14058A00E9D5089503D6B8016030E0E07E071CF44EEC5FEF03
:14059E0002C042E350E08B01040F151F24E630E01DD59801BA
:1405B20004E610E0BFD5A80140555B4F24E630E08A0112D553
:1405C600A80120E832E00AD528E230E00BD5602F20E530E0E1
:1405DA008A0102D525E030E003D5A02E2AE030E08A01FAD47D
:1405EE00402F88E290E0E62FFF27E80FF91F6491EA2DFF2734
:14060200E80FF91FA49088E390E0E42FFF27E80FF91F4491A9
:140616002A2C220C220C220C242A209428BA609545B3487F58
:14062A00862F8770482B45BB93D50895CAD580916000909167
:14063E006100019690936100809360008330E0E09E0769F444
:140652000AE010E089DEAB9889B78E7F89BF2224332430921C
:14066600610020926000C6D51895B3D497D569970024112479
:14067A001D8A0C8A8BC4EDA1FEA18081853251F00081EBA1AD
:14068E00FCA18BD58C899D8901969D8B8C8B77C400241124B6
:1406A2001B8A0A8A8FEF9FEF9F8B8E8B198A088A83E291E0B1
:1406B6009D838C8380E2888F8DA19EA101969EA38DA3CC2423
:1406CA00DD24EDA1FEA1208033243F862E86822D932D80325D
:1406DE00E0E09E0759F18332E0E09E0799F08032E0E09E079F
:1406F2008CF18E859F858B32E0E09E07A9F08D32E0E09E0761
:1407060059F08033E0E09E07E9F022C0888999898160998B8B
:14071A00888B20C0888999898460998B888B1AC0888999897D
:14072E008860998B888B8BE2888F12C0888999898860998B03
:14074200888B80E2888F0AC0888999898061998B888B04C03E
:1407560081E090E0C82ED92ECC2011F4DD2009F006C08DA1E6
:14076A009EA101969EA38DA3ACCFEDA1FEA100811127D6D627
:14077E0000300107A1F00DA11EA18ED51B8B0A8B05C08DA1A0
:140792009EA101969EA38DA3EDA1FEA100811127C3D600305D
:1407A600010799F716C0EDA1FEA180818A3289F48FA198A5FD
:1407BA00029698A78FA3E82FF92F3297208031803B8A2A8A50
:1407CE008DA19EA101969EA38DA3EDA1FEA180818E3209F0BB
:1407E20037C08E2F9F2F01969EA38DA3E82FF92F0081112781
:1407F60099D600300107A1F00DA11EA151D51F8B0E8B05C01C
:14080A008DA19EA101969EA38DA3EDA1FEA10081112786D623
:14081E000030010799F716C0EDA1FEA180818A3289F48FA191
:1408320098A5029698A78FA3E82FF92F3297208031803F8A4A
:140846002E8A8DA19EA101969EA38DA3EDA1FEA180818C3681
:14085A0051F48E2F9F2F01969EA38DA3888999898260998B79
:14086E00888BEDA1FEA1208033243F862E86822D932D88359A
:14088200E0E09E0709F4D0C088E582159305A4F08E859F8509
:140896008534E0E09E0709F471C38534E0E09E070CF43EC0E3
:1408AA008E859F858335E0E09E0709F4C8C136C08E859F8533
:1408BE008F36E0E09E0709F4B1C08FE690E02E843F8482159D
:1408D2009305B4F08E859F858336E0E09E0709F48CC184367D
:1408E600E0E09E0749F18536E0E09E0709F446C38636E0E0BD
:1408FA009E0709F441C312C08E859F858337E0E09E0709F41F
:14090E0067C28537E0E09E0709F488C08837E0E09E0709F425
:1409220083C000C0EDA1FEA10081EBA1FCA13BD48C899D899D
:1409360001969D8B8C8B27C30888198801FE47C08FA198A549
:14094A00049698A78FA3E82FF92F349720803180428053809E
:14095E00EC2FFD2F208631864286538640E050E060E070E060
:14097200EC2FFD2F2084318442845384241635064606570616
:14098600A4F4888999898860998B888B8DE2888FEC2FFD2FA6
:14099A0000851185228533850BD4EC2FFD2F008711872287E1
:1409AE0033878AE090E09B838A83EC2FFD2F20843184428410
:1409C200538448825982222D332D0C811D8113D5EFC08FA104
:1409D60098A5029698A78FA3E82FF92F3297208031803F82AD
:1409EA002E82822D932D8030E0E09E077CF48889998988603A
:1409FE00998B888B8DE2888F8E819F81809590958F5F9F4FE3
:140A12009F838E838AE090E0998388832E813F810C811D8102
:140A26008DD4C4C00888198801FE13C08FA198A5049698A78E
:140A3A008FA3E82FF92F34972080318042805380EC2FFD2F3F
:140A4E0020863186428653860CC08FA198A5029698A78FA354
:140A6200E82FF92F3297208031803F822E82EDA1FEA1808188
:140A7600853701F50888198801FE12C08AE090E09B838A83B3
:140A8A00EC2FFD2F208431844284538448825982222D332DC7
:140A9E000C811D81AAD486C08AE090E0998388832E813F81E5
:140AB2000C811D8145D47CC0EDA1FEA180818F3651F50888E7
:140AC600198800FE06C080E3EC81FD818193FD83EC830888D6
:140ADA00198801FE12C088E090E09B838A83EC2FFD2F2084A8
:140AEE0031844284538448825982222D332D0C811D817BD4D4
:140B020057C088E090E0998388832E813F810C811D8116D445
:140B16004DC00888198800FE0EC080E3EC81FD818193FD83DF
:140B2A00EC83EDA1FEA12080EC81FD812192FD83EC8308885E
:140B3E00198801FE12C080E190E09B838A83EC2FFD2F20844A
:140B520031844284538448825982222D332D0C811D8149D4A1
:140B660009C080E190E0998388832E813F810C811D81E4D369
:140B7A00EDA1FEA180818835B9F483E291E0E82EF92E0DC0EF
:140B8E00EE2DFF2D00811127F3D4EE2DFF2D00838E2D9F2D3B
:140BA2000196E82EF92EEE2DFF2D2080222071F783E291E004
:140BB600E82EF92E8E899F898F3FEFEF9E0721F400241124F0
:140BCA001F8A0E8A0E881F88002019F4112009F413C103E285
:140BDE0011E0EFD11F830E83202E312E0E881F880016110608
:140BF2000CF006C13F8A2E8A03C18FA198A5029698A78FA371
:140C0600E82FF92F3297208031802C8681E090E00A881B88C9
:140C1A008015910554F41F8A0E8A22242D868C2F9D2F0C96F0
:140C2E00E82EF92EE7C00C85EBA1FCA1B6D28C899D890196BA
:140C42009D8B8C8BA2C18FA198A5029698A78FA3E82FF92F47
:140C56003297A080B1808E899F898F3FEFEF9E0721F40024A7
:140C6A0011241F8A0E8A0A881B88002011F4112049F00A2D05
:140C7E001B2D05D34A885B88401A510A5B8A4A8A0E881F88E2
:140C9200002039F4112029F40A2D1B2DF6D21F8B0E8B0A8897
:140CA6001B88002011F4112049F00888198803FE05C08A89FE
:140CBA009B8901979B8B8A8B0888198804FE26C003FE09C04C
:140CCE00088DEBA1FCA169D28C899D8901969D8B8C8B088878
:140CE200198802FC50C00EC000E3EBA1FCA15BD28C899D890D
:140CF60001969D8B8C8B8A899B8901979B8B8A8B222433246D
:140D0A000A881B88201431045CF339C00888198802FC16C0EA
:140D1E000EC000E2EBA1FCA140D28C899D8901969D8B8C8BC5
:140D32008A899B8901979B8B8A8B222433240A881B8820149D
:140D460031045CF30888198803FE1BC0088DEBA1FCA127D251
:140D5A008C899D8901969D8B8C8B11C0EA2DFB2DC895002DDA
:140D6E00EBA1FCA11AD28C899D8901969D8B8C8B8A2D9B2DCC
:140D82000196A82EB92EEA2DFB2DC895002059F02E883F8887
:140D9600822D932D01979F8B8E8B222009F73320F9F60888EB
:140DAA00198802FEEEC00EC000E2EBA1FCA1F7D18C899D890A
:140DBE0001969D8B8C8B8A899B8901979B8B8A8B22243324A4
:140DD2000A881B88201431045CF3D7C08FA198A5029698A745
:140DE6008FA3E82FF92F3297E080F180EE2031F4FF2021F487
:140DFA008BEE90E0E82EF92E8E899F898F3FEFEF9E0721F41A
:140E0E00002411241F8A0E8A0A881B88002011F4112049F072
:140E22000E2D1F2DCCD04A885B88401A510A5B8A4A8A0E88E0
:140E36001F88002039F4112029F40E2D1F2DBDD01F8B0E8B0F
:140E4A000A881B88002011F4112049F00888198803FE05C0D9
:140E5E008A899B8901979B8B8A8B0888198804FE26C003FE5C
:140E720009C0088DEBA1FCA196D18C899D8901969D8B8C8B6D
:140E86000888198802FC4FC00EC000E3EBA1FCA188D18C89D2
:140E9A009D8901969D8B8C8B8A899B8901979B8B8A8B2224F8
:140EAE0033240A881B88201431045CF338C00888198802FCC5
:140EC20016C00EC000E2EBA1FCA16DD18C899D8901969D8B35
:140ED6008C8B8A899B8901979B8B8A8B222433240A881B8815
:140EEA00201431045CF30888198803FE1AC0088DEBA1FCA172
:140EFE0054D18C899D8901969D8B8C8B10C0EE2DFF2D008112
:140F1200EBA1FCA148D18C899D8901969D8B8C8B8E2D9F2DF1
:140F26000196E82EF92EEE2DFF2D2080222059F02E883F88F4
:140F3A00822D932D01979F8B8E8B222011F7332001F7088834
:140F4E00198802FE1CC00EC000E2EBA1FCA125D18C899D8908
:140F620001969D8B8C8B8A899B8901979B8B8A8B22243324FE
:140F76000A881B88201431045CF305C080EC90E0E82EF92E9C
:140F8A003BCF8DA19EA101969EA38DA3EDA1FEA120802220C5
:140F9E0009F06FCB0C891D896996DAD024960895A02FB12F22
:140FB200E22FF32F01900D920020E1F70895E02FF12FAA2733
:140FC600BB270190002011F01196FBCF0A2F1B2F08953A9325
:140FDA002A931A930A9308956894DA92D12E04C0E894DA924C
:140FEE00D12ED32617FF04C0109500950F5F1F4F37FF04C00D
:14100200309520952F5F3F4F0BD0D7FE04C0109500950F5F28
:141016001F4FD9900895689401C0E894EA92FA928A93EE24E2
:14102A00FF2480E1000F111FEE1CFF1CE216F30618F0E21AD5
:14103E00F30A03958A95A1F716F40E2D1F2D8991F990E990A5
:141052000895E89401C068942FD0CC2408C0E89401C06894C4
:1410660029D037FD53D0B7FD5AD0772488249924AA24BB2497
:14107A0041D0C1F044D0B1F0E8E2000F111F221F331F771CBC
:14108E00881C991CAA1CBB1C88169906AA06BB0628F0881AF0
:1410A200990AAA0ABB0A0395EA9559F726F4082D192D2A2DCB
:1410B6003B2D13C07A928A929A92AA92BA92CA92EA938A9319
:1410CA009A93AA93BA938B859C85AD85BE85C32E0EF0CB26D5
:1410DE000895C7FC17D0B991A99199918991E991C990B990D3
:1410F200A99099908990799024960895E02FE12BE22BE32BD9
:141106000895E82FE92BEA2BEB2B0895009510952095309591
:14111A000F5F1F4F2F4F3F4F089580959095A095B0958F5F9A
:14112E009F4FAF4FBF4F08950A921A928A939A93029FC00122
:14114200129F900D039F900D8C01999189911990099008955C
:14115600E2E008C0E4E006C0EE2704C05A934A930895E1E070
:14116A0049915991E0FD089569917991E1FD0895A990B99032
:14117E00E2FD0895C990D990E3FD0895E990F99008957A93F6
:141192006A93E6CFBA92AA92FACFDA92CA92FACFFA92EA92AD
:1411A600FACF0A92C8950A923196C895F02DE99109900994E6
:1411BA0000951095209530950F5F1F4F2F4F3F4F0895FA935B
:1411CE00EA93BA93AA939A938A933A932A931A930A939A92BC
:1411E2008A927A926A925A924A923A922A921A920A920FB678
:1411F6000A92089509900FBE099019902990399049905990C0
:14120A00699079908990999009911991299139918991999180
:14121E00A991B991E991F99108950A921A92002411240030C6
:14123200010741F01695079510F4020E131E220F331FF5CF9C
:14124600002D112D19900990089588DF402F20903C013090C7
:14125A003D01222011F4332021F04A3011F40DE0F2DF5D9B62
:14126E00FECF4CB9042F112778DF0895822F932F01968E7F24
:14128200800F911F082F192F0895E02FF12FAA27BB27C895BE
:14129600002019F031961196FACF0A2F1B2F089577DF602FDF
:1412AA00712F02C06F5F7F4FE62FF72F0081112753D10030EA
:1412BE000107B1F7AA24BB24E62FF72F80818D3239F481E036
:1412D20090E0A82EB92E6F5F7F4F07C0E62FF72F80818B327F
:1412E60011F46F5F7F4F4427552711C00AE010E0242F352F0A
:1412FA0096DF402F512FE62FF72F21906E2F7F2F3324420D9F
:14130E00531D40535040E62FF72F0081112706D10030010735
:1413220039F7AA2011F4BB2039F0042F152F009510950F5F95
:141336001F4F02C0042F152F0DDF08952FDFC22ED32E402F05
:14134A00512F2B97AD88BE88CC2029F4DD2019F464E071E02A
:14135E0044C022242A866C2F7D2F665F7F4F37C02A2D3B2DF1
:141372000C2D1D2D52DEE02EF12E0A30E0E01E0774F4862F4B
:14138600972F0197282E392E682F792F8E2D9F2DC096E22D0D
:14139A00F32D808317C08A2D9B2D8031E0E09E0789F4862F7E
:1413AE00972F0197282E392E682F792F83EF90E0EE2DFF2DA8
:1413C200E80FF91F4080E22DF32D40822A2D3B2D0C2D1D2D15
:1413D60024DEC02ED12ECC2009F0C6CFDD2009F0C3CF262FBD
:1413EA00372F042F152FDEDD2B96B4DE0895EFDDD3DE6A97E9
:1413FE00CAA4DBA440E050E060E070E0EC2FFD2F26A037A02A
:1414120040A451A4241635064606570629F48DE091E0E82EBE
:14142600F92E77C02224298E8C2F9D2F4996E82EF92E5FC095
:14143A002C2C3D2C442437FC4094552447FC5094EC2FFD2F87
:14144E0066A077A080A491A45A924A923A922A92062D172D4D
:14146200282D392DF8DDA02EB12E0A30E0E01E0774F48E2DF7
:141476009F2D0197282E392EE82EF92E8A2D9B2DC096E22D20
:14148A00F32D808317C08C2D9D2D8031E0E09E0789F48E2D83
:14149E009F2D0197282E392EE82EF92E8CEF90E0EA2DFB2DB2
:1414B200E80FF91F4080E22DF32D40822C2C3D2C442437FC0A
:1414C6004094552447FC5094EC2FFD2F66A077A080A491A4E1
:1414DA005A924A923A922A92062D172D282D392DB4DDEC2FD0
:1414EE00FD2F06A317A320A731A740E050E060E070E0EC2FC1
:14150200FD2F26A037A040A451A4241635064606570609F01C
:1415160091CF2E2D3F2D0CA11DA146DD6A961CDE24960895BB
:14152A0083E490E0202E312E280E391EE22DF32DC895002DE3
:14153E00112704701070089583E490E0202E312E280E391EBF
:14155200E22DF32DC895002D112702701070089583E490E02E
:14156600202E312E280E391EE22DF32DC895002D11270071D5
:14157A0010700895F1DD402F512F042F152FDEDF0030010717
:14158E0039F0042F152F015610400F5B1F4F02C0042F152FF1
:1415A200E2DD089518DDDCDD229722E030E00C2F1D2F0C5F6E
:1415B6001F4F60DE402F512F598348832C813D8106E210E09C
:0E15CA0052D8402F512F2296CADD2496089544
:00000001FF
